:100000000C9462000C94BB1A0C94E81A0C948A00AD
:100010000C948A000C948A000C948A000C948A0038
:100020000C948A000C948A000C948A000C948A0028
:100030000C948A000C948E0B0C948A000C948A0009
:100040000C94151B0C948A000C94911E0C94D41ED5
:100050000C948A000C948A000C948A000C948A00F8
:100060000C94EF080C948A000000000700020100C5
:100070000003040600000000000000000102040864
:100080001020408001020408102001020408102002
:10009000040404040404040402020202020203032E
:1000A00003030303000000002300260029000000D2
:1000B0000000250028002B0000000000240027007D
:1000C0002A00C21F11241FBECFEFD8E0DEBFCDBF74
:1000D00012E0A0E0B1E0E8EFF1E402C005900D927B
:1000E000A23EB107D9F714E0A2EEB2E001C01D9222
:1000F000AC3CB107E1F710E0C4ECD0E004C02297BB
:10010000FE010E94D720C23CD107C9F70E94FE1F02
:100110000C94FA200C9400008091CE03813019F4E5
:1001200082E08093CE038091CE03833019F484E083
:100130008093CE030895A8950895CF93DF93FC0193
:10014000962F9270862F817060FF20C0992331F026
:100150008091600380831092E20216C0A091E202B7
:10016000C091F903C770D0E0CA56DD4F8881A81747
:1001700010F080E03CC081E08A0F8093E202B0E0A2
:10018000A05FBC4F8C91808381E031C09923C1F086
:1001900090819093E3021092E202292F207E203674
:1001A00051F490916003923020F390819F7190936D
:1001B000A20393E01AC09E3F39F71092600317C064
:1001C0009091E3029F3F01F79091E202993288F605
:1001D00021E0290F2093E2023081E92FF0E0EF5275
:1001E000FC4F3083293281F691E090936003DF91D8
:1001F000CF910895DC01ED91FC910190F081E02D0B
:1002000009950895DC01ED91FC910190F081E02DBC
:10021000099508952091CF033091D003382748E005
:10022000C901880F991F37FF06C09C0151E225279D
:1002300050E1352701C09C01415091F73093D00324
:100240002093CF0308958436910520F4BC0180E00B
:1002500090E017C09C018E3B910528F42A55310986
:10026000AAE0B0E00CC0823D910528F4245B31097E
:10027000A4E6B0E004C02D5C3109A8E5B2E00E941C
:100280000B20A4E6B0E09B01AC010E941A20089567
:1002900090E08C599F4F0E942301089581E0809344
:1002A000FA0391E29093FB031092FC038093FD0309
:1002B00082E08093FE0383E08093FF0384E08093D9
:1002C000000485E08093010486E08093020487E0C7
:1002D0008093030486E2809304048093050484E2FF
:1002E0008093060485E280930704089560E08EE021
:1002F0000E94231C61E08FE00E94231C61E080E1EA
:100300000E94231C60E082E00E94231C61E084E0E4
:100310000E94231C089542E050E06CE870E080E009
:100320000E949B1A0895E3E0F0E089E08093570073
:10033000E491E67081E0E63009F080E00895CF9323
:10034000DF93C82F0E949301882381F0DFB781E0FB
:100350008093CD03F8940E949B0088E18093600015
:10036000C0936000C1110E949B00DFBFDF91CF915D
:100370000895FC0140A5842F877090E0959587959E
:100380000196242F217030E0820F931F880F880F71
:1003900008958F929F92AF92BF92CF92DF92EF9289
:1003A000FF92CF93FC01C0A5EC2FE770F0E0EA5676
:1003B000FD4FA081B0E0C7FF03C024E130E002C0E0
:1003C0002FE030E0FC0197A183E1989FF001112418
:1003D000E65AFE4F80809180A280B380A20FB31FA7
:1003E00020E43FE14DE750E00E942520A501940163
:1003F0000E945D208C2F887149F469017A01E0ED3B
:10040000CE0EE7E0DE1EE11CF11C1BC0C7FF05C0DD
:1004100060E47AE88CE29EE004C060E07EEE8AEB65
:100420009BE069017A01F8EBCF0EFBE0DF1EE11CD7
:10043000F11CA50194010E945D20C20ED31EE41E92
:10044000F51EC701B60169517C4F8F4F9F4F28EEB3
:1004500033E040E050E00E945D20A8EEB3E00E944F
:100460001A20CF91FF90EF90DF90CF90BF90AF9088
:100470009F908F900895DB01FA01582F569590E0D8
:100480002481237030E0322F22274081240F311D38
:1004900011963C932E9344814C70218130E060E4AE
:1004A000469F200D311D112413963C932E931297D5
:1004B00044814073228130E060E1469F200D311D70
:1004C000112415963C932E9314974481407C2381EC
:1004D00030E064E0469F200D311D112417963C93B7
:1004E0002E931697359618969F5F591748F680FFFA
:1004F00047C0408142954695469543702DE431E0D2
:10050000429FC001439F900D11240C9611969C931D
:100510008E93808190E074E0969587957A95E1F7C7
:1005200083709927829FA001839F500D929F500D49
:100530001124445F5F4F13965C934E931297808112
:1005400090E0969587959695879583709927829FD9
:10055000A001839F500D929F500D1124445F5F4F67
:1005600015965C934E93149740814370429FC0014F
:10057000439F900D11240C9617969C938E9316977B
:100580000895803223E0920708F1883E23E0920725
:1005900040F48F519340E4E096958795EA95E1F712
:1005A0000895803D27E0920718F48C5D93400895EC
:1005B000883928E0920768F4885C974074E0969543
:1005C00087957A95E1F78D509C4F089580E090E0F3
:1005D00008958FEF93E008958C30910540F4A4E0E6
:1005E000880F991FAA95E1F7885D9C4F0895843F75
:1005F00023E0920718F484529C4F0895811524E05B
:10060000920740F48657934FF4E0880F991FFA95AC
:10061000E1F7089580E998E008959C0136952795C3
:1006200025753575821B930B9C0123733373969547
:1006300087959695879583739373820F931F9C017B
:1006400054E0369527955A95E1F7280F391F2F70FA
:100650003F7041E051E0249FC001259F900D349FE1
:10066000900D1124892F08954298882319F00000D5
:10067000419A02C0000041980000429A000008958B
:10068000429A000086B14298000081700895CF938D
:10069000DF93D82F5C9A42985C98C8E08D2F8078C1
:1006A0000E943403DD0FC150C9F74298DF91CF910A
:1006B00008958F770E9447030895CF93DF93D82F33
:1006C000C8E08D2F80780E943403DD0FC150C9F738
:1006D0004298DF91CF910895CF93DF934298C8E07D
:1006E00080E0D82FDD0F0E9440038D0FC150C9F765
:1006F000DF91CF9108950E9459030E946C035C9A88
:100700000895A1E0B0E0E7E8F3E00C94AE20806843
:1007100069830E9447036981862F0E945D035C9A6A
:100720002196E2E00C94CA20CF93C091DA03C82747
:10073000E82FF0E0EF52FC4F678589E70E948103C4
:100740006C2F8DE30E9481036C2F82E40E94810351
:10075000CF91089586E20E947B030895CF938BE2A8
:100760000E947B03C82F8CE20E947B03282F30E07D
:1007700066E0369527956A95E1F744E0C49FC0018D
:100780001124822B932BCF910895CF93DF93EC010B
:100790006C818CE10E9481036D818DE10E94810357
:1007A0006E818EE10E9481036F8180E20E9481034D
:1007B000688581E20E948103698582E20E9481034B
:1007C0006A8583E20E9481036B8584E20E94810333
:1007D0006C8585E20E9481036D858AE20E94810317
:1007E0006E858EE60E9481036F858FE60E948103ED
:1007F000688980E70E948103698981E70E948103FB
:100800006A8982E70E948103DF91CF910895CF9298
:10081000DF92EF92FF92CF93DF936B017C01C114C3
:1008200088E3D8068CE9E8068CE1F80628F5C701CC
:10083000B60120E836E948E950E00E945D20E90170
:10084000689760E879E687E69FEF0E942D206C0D9F
:100850007D1D8E1D9F1DF2E0660F771F881F991F5B
:10086000FA95D1F721E732E040E050E00E945D20A8
:10087000F22EE32E80E421C0C701B60120E03DE264
:1008800041E351E00E945D20E901689760E073ED6B
:100890008EEC9EEF0E942D206C0D7D1D8E1D9F1DE8
:1008A000660F771F881F991F21E732E040E050E074
:1008B0000E945D20F22EE32E80E66C2F6F71680F90
:1008C00085E70E9481036E2D86E70E9481036F2DCC
:1008D00087E70E948103DF91CF91FF90EF90DF9037
:1008E000CF9008958F929F92AF92BF92CF92DF9256
:1008F000EF92FF92CF93DF93D82F83E00E947B0388
:100900008093CC0384E00E947B038093CB0360E060
:1009100086E00E94810361E087E00E9481036FE727
:1009200089E00E94810365E08AE00E94810362E120
:100930008BE00E94810365E18CE00E9481036DEFF2
:100940008DE00E94810360E08EE00E948103DD2340
:1009500019F087E491E008C02091F80333E1239F68
:10096000C0011124865A9E4F0E94C5036CE880E3A3
:100970000E9481036FE082E30E94810362E483E3CB
:100980000E9481038091F90387FF02C064E101C0E6
:100990006AE084E30E9481036AE285E30E948103A6
:1009A0006DE286E30E94810364ED87E30E94810388
:1009B00060E088E30E94810360E089E30E94810394
:1009C000D11109C0C090DA03D090DB03E090DC03C2
:1009D000F090DD0307C0C5E9CC2EC1ECDC2EED2C78
:1009E000CEEDFC2ECAE38F2C9924AA24BB24682DBB
:1009F0008C2F0E948103682D85E08C0F0E9481035B
:100A0000FE2CED2CDC2CCC24CF5FCE3361F76FEFC6
:100A100083E40E9481036FEF84E40E9481036FEFFF
:100A200085E40E9481036FEF86E40E948103DD2349
:100A300011F066E002C06091DE038DE60E94810342
:100A400060E089E70E9481036091DF038AE70E94EA
:100A5000810360E083E70E94810360E084E70E94F5
:100A60008103D11109C06091D6037091D7038091A1
:100A7000D8039091D90304C060EC7AEC89E896E33E
:100A80000E940704DF91CF91FF90EF90DF90CF900D
:100A9000BF90AF909F908F90089561E087E00E9493
:100AA000810364E28EE70E94810363E088E00E9494
:100AB000810360E088E00E94810365E087E00E9496
:100AC000810362E085E00E94810383E00E947B0352
:100AD0008093CC0384E00E947B038093CB03089532
:100AE00083E00E947B038093CC0384E00E947B031D
:100AF0008093CB0361E087E00E9481036AE070E0AD
:100B000080E090E00E948E1B0E944D050000089539
:100B1000CF92DF92FF920F931F93CF93DF931F9299
:100B2000CDB7DEB7082F162F8EE399830E9481037D
:100B3000F02EC02E9981D92E8C2D8F19811738F463
:100B4000F60161916F018FE70E948103F5CF64E0A8
:100B500085E00E94810383E00E947B038093CC03A5
:100B600084E00E947B038093CB030E946B1B609305
:100B7000C7037093C8038093C9039093CA0369E0C5
:100B800087E00E94810381E08093CE030F90DF9184
:100B9000CF911F910F91FF90DF90CF9008950F9309
:100BA0001F930E9488058091CE03813099F40E94A2
:100BB0006B1B0091C7031091C8032091C9033091AA
:100BC000CA03601B710B820B930B603A764881401D
:100BD000910548F38091CE03813031F46AEB71E0E6
:100BE00082E294E00E942D1D1F910F9108950F93B2
:100BF0001F938091CE03823021F41092CE0381E0C6
:100C000020C08091CE038130D9F40E946B1B0091EB
:100C1000C7031091C8032091C9033091CA03601B18
:100C2000710B820B930B613A76488140910540F03D
:100C300061E087E00E9481031092CE0382E001C050
:100C400080E01F910F910895EF92FF920F931F93F1
:100C5000CF93DF938B019C01442737FD4095542FA0
:100C600060E271EA87E090E00E947F20E9011C16B3
:100C70001D0614F0C1E0D0E0D80120E231EA47E0DF
:100C800050E00E9425209E01442737FD4095542FB7
:100C90000E947F20790100E010E00E151F055CF432
:100CA000419ACE010E94B41B4198CE010E94B41B10
:100CB0000F5F1F4FF2CFCDB7DEB7E6E00C94C62032
:100CC000CF93DF932D9A60910A0470910B04809169
:100CD0000C0490910D040E94070460E089E70E94D3
:100CE000810361E070E080E090E00E948E1B0E9432
:100CF000AA03C82F61E070E080E090E00E948E1BA4
:100D00000E94AA03D0E0C80FD11D61E070E080E02E
:100D100090E00E948E1B0E94AA03C80FD11D61E0C3
:100D200070E080E090E00E948E1B0E94AA032D9844
:100D30009E01280F311DC901969587959695879537
:100D4000DF91CF910895CF93C82F2D9A83E00E9411
:100D50007B038093CC0384E00E947B038093CB03CE
:100D600060E086E00E94810361E087E00E948103E9
:100D70006FE789E00E94810365E08AE00E948103B9
:100D800062E18BE00E94810365E18CE00E948103B7
:100D90006DEF8DE00E94810360E08EE00E94810390
:100DA0006CE280E70E94810360E080E30E9481039F
:100DB00060E089E70E94810365E08AE70E94810381
:100DC00062E181E70E94810362E082E70E94810381
:100DD00060E083E70E94810360E084E70E94810372
:100DE00060910A0470910B0480910C0490910D04A1
:100DF0000E94070467E08DE60E9481036AE070E0CC
:100E000080E090E00E948E1B69E087E00E948103F1
:100E10006AE070E080E090E00E948E1BCC2369F0D5
:100E2000C5E1C15009F459C061E070E088EB91E080
:100E30000E9424060E949B00F4CF61E070E088E8E5
:100E400091E00E9424060E949B0065E08DE60E94CE
:100E500081036AE070E080E090E00E948E1B61E018
:100E600070E088EB91E00E9424060E949B0064E001
:100E70008DE60E9481036AE070E080E090E00E94CD
:100E80008E1B61E070E08DE591E00E9424060E94D7
:100E90009B0062E08DE60E9481036AE070E080E0E2
:100EA00090E00E948E1B61E070E08FEA90E00E946B
:100EB00024060E949B0060E08DE60E9481036AE0A8
:100EC00070E080E090E00E948E1B62E070E085E0C0
:100ED00091E00E9424060E949B0061E087E00E944E
:100EE00081032D98CF910895CF93DF93EC014AE0D1
:100EF00050E06D2F70E082E294E00E94F21D6EE2FD
:100F000082E294E00E94111DBE0184E0769567950F
:100F10008A95E1F76F7077274AE050E082E294E02B
:100F20000E94F21DDF91CF910895D82FC0E0CD1718
:100F300080F4439A64E670E080E090E00E948E1BAB
:100F4000439864E670E080E090E00E948E1BCF5FE3
:100F5000EECF6CE271E080E090E00E948E1BE6CF65
:100F60000F931F93CF93DF93EC01062F15E01150E1
:100F700051F0CE010E94E420081741F0602FCE010D
:100F80000E94EC20F4CF82E00E949507DF91CF9180
:100F90001F910F910895A0E0B0E0E1EDF7E00C940F
:100FA000A020482E562EC0E0D0E0612C712CE12C00
:100FB000F12C00E010E0442079F081E04816A1F027
:100FC00092E0491219C028E4622E712C30E2E32E1F
:100FD000F12C03E613E010C0612C712C6BE1E62EBE
:100FE000F12C0AEF13E008C04DE1642E712C59E298
:100FF000E52EF12C01ED13E043018C0E9D1E1092A5
:10100000D0031092CF033401A62CA818B12CC30131
:1010100001966C01AE14BF04A8F4A00EB11E5110CD
:1010200006C0C3010E94E420F501808305C0F501DC
:101030006081C3010E94B007F50180810E940A010E
:101040003601E2CFC301511018C0C3010E94E42051
:10105000B82EC6010E94E4202B2D30E0322F22272B
:10106000282B8091CF039091D0038217930779F4B6
:10107000C0E0D0E0552453949ECF36016091D00358
:101080000E94B0076091CF03C6010E94B007D395BC
:10109000C13093E0D90708F48ECF852DCDB7DEB7E8
:1010A000E0E10C94BC2060E081E00E94CB07882343
:1010B00031F081E09091D103983309F080E00895F8
:1010C00061E081E00E94CB07089561E082E00E9428
:1010D000CB07089560E082E00E94CB07811108C031
:1010E000E3E6F3E01192119283E0E338F807D1F7D9
:1010F0000895A1E0B0E0EFE7F8E00C94AE2089831A
:101100000E944E0192E0909308049FEF909309048F
:101110009AE0909312041092130410921404109207
:101120000A0410920B0410920C0410920D042EE18C
:1011300020930E0490930F0428EB3BE030931104AE
:10114000209310048981882371F061E080E00E947F
:10115000CB07E3E6F3E01192119283E0E338F8075E
:10116000D1F70E9465082196E2E00C94CA2060E065
:1011700080E00E94CB07811103C081E00E947908C2
:101180000895CF93C1E0811101C0C0E06C2F82E1CE
:101190000E945C1C6C2F83E10E945C1C1092C103B6
:1011A0001092C0038091B9008C6F8093B90080E2E7
:1011B0008093B80085E48093BC00CF91089585EDBD
:1011C0008093BC008091BC0084FDFCCF0895ECEBC3
:1011D000F0E0108285E480831092C00308951F928E
:1011E0000F920FB60F9211242F933F934F935F935B
:1011F0006F937F938F939F93AF93BF93EF93FF93DF
:10120000CF93DF931F92CDB7DEB78091B900887F6F
:10121000803609F4C7C0A8F5883209F464C098F490
:10122000803109F45DC038F4882309F4F3C08830B4
:1012300009F456C0F1C0883109F455C0803209F074
:10124000EBC082E0A7C0803409F477C078F4803323
:1012500009F45FC0883309F0DFC084E08093BF03E6
:101260008091C0038B7F8093C003D0C0803509F488
:1012700052C0883509F467C0883409F0CDC085E0D4
:1012800089C0883909F4C0C0A8F4883709F48AC035
:1012900038F4883609F486C0803709F483C0BCC0AE
:1012A000883809F4B1C0803909F47FC0803809F06A
:1012B000B3C07BC0803B09F493C038F4803A09F492
:1012C0008CC0883A09F48CC0A7C0803C09F49EC049
:1012D000883C09F49BC0883B09F09EC080E081C037
:1012E0008091C40313C08091C1039FEF980F909326
:1012F000C1038823D1F1E091C203F091C303CF0170
:1013000001969093C3038093C20380818093BB00B6
:101310007DC083E03FC0E091C203F091C303CF01E1
:1013200001969093C3038093C2038091BB00808396
:101330008091C10381508093C1038091C1038230A9
:1013400008F064C061C0E091C203F091C303CF0113
:1013500001969093C3038093C2038091BB00808366
:101360008091C10381508093C1038091C0038B7F22
:101370008093C0038091C00380FF4CC08091C00364
:101380008E7F8093C0038091C00382608093C003EE
:1013900084EA3DC08093BF038091C0038B7F80931C
:1013A000C00338C01092C10331C0E091C503F09171
:1013B000C603309749F18091BB0089838091C103B6
:1013C00091E0980F9093C103811102C062E001C0C7
:1013D00060E0CE010196099515C00E94DF0816C095
:1013E00081E0E091C503F091C603309769F088234E
:1013F00011F063E001C061E0CE0101960995998189
:101400009093BB00811102C085E801C085EC8093F8
:10141000BC0002C00E94DF080F90DF91CF91FF91C6
:10142000EF91BF91AF919F918F917F916F915F915C
:101430004F913F912F910F900FBE0F901F901895D5
:101440008F929F92AF92BF92CF92DF92EF92FF92D4
:10145000CF93DF93EC010E946B1B6B017C014E016B
:10146000A12CB12C8091C00382FF11C02097D1F331
:101470000E946B1B6C197D098E099F0986169706C1
:10148000A806B90678F70E94E70881E004C08091B9
:10149000BF031092BF03DF91CF91FF90EF90DF90D9
:1014A000CF90BF90AF909F908F900895A2E0B0E052
:1014B000ECE5FAE00C94AA20182F7B01022F0470AF
:1014C00022FD05C080910B0190910C0102C080E0CB
:1014D00090E02A8349830E94200A2A814981811150
:1014E00036C01092BF034093C103F092C303E09251
:1014F000C203110F1093C4039091C00321FF02C0D7
:1015000085E001C084E0892B8093C0038091C003F3
:1015100081FF0BC08091C0038D7F8093C0038091B9
:10152000C4038093BB0085EC01C085EE8093BC00B2
:10153000822F817020FF0BC0011105C080910B012B
:1015400090910C0102C080E090E00E94200A229657
:10155000E6E00C94C620A2E0B0E0E1EBFAE00C94E7
:10156000AA20182F7B01022F047022FD05C0809154
:101570000B0190910C0102C080E090E02A83498326
:101580000E94200A2A814981811138C01092BF032C
:101590004093C103F092C303E092C203812F880FEE
:1015A00081608093C4039091C00321FF02C085E055
:1015B00001C084E0892B8093C0038091C00381FF28
:1015C0000BC08091C0038D7F8093C0038091C403C2
:1015D0008093BB0085EC01C085EE8093BC00822F18
:1015E000817020FF0BC0011105C080910B0190910B
:1015F0000C0102C080E090E00E94200A2296E6E002
:101600000C94C620A0E0B0E0E8E0FBE00C94A82039
:101610000E946B1B0091BB031091BC032091BD0382
:101620003091BE036B017C01C01AD10AE20AF30AB1
:101630009701860141E1C41647E2D406E104F104B2
:1016400008F442C02091BA0331E0320F3093BA035C
:1016500020FF02C017E001C010E06093BB0370934D
:10166000BC038093BD039093BE0363E070E082E20D
:1016700094E00E94020161E070E082E294E00E9446
:10168000020107E0010F812F90E0EC01CC0FDD1F7C
:10169000C35FDE4F68817981672F77276370772773
:1016A000880F991F880F991F682B792B82E294E08D
:1016B0000E94FA0068817981772782E294E00E9493
:1016C000FA001F5F1013DFCFCDB7DEB7E8E00C9450
:1016D000C42025B190E0FC01EE0FFF1FE80FF91FB9
:1016E000E65DFC4F8081282B25B988B19181892B3B
:1016F00088B98BB19281892B8BB9089585B190916E
:101700002703892385B988B190912803892388B953
:101710008BB19091290389238BB908951F920F9261
:101720000FB60F9211242F933F934F935F936F93B4
:101730007F938F939F93AF93BF93CF93EF93FF9339
:10174000C091860380910601C81708F03EC08091C1
:101750002503909126039093870080938600EC2FB9
:10176000F0E0EE0FFF1FE35FFE4F808191810E944A
:10177000EC02880F991F9093260380932503809194
:101780002503909126032091070130910801281B21
:10179000390B309308012093070180911004909138
:1017A0001104880F991F2817390720F49093080116
:1017B0008093070180918403811142C080910804C5
:1017C00080FF41C0C830E0F53EC080912503909174
:1017D0002603909387008093860080910701909163
:1017E0000801909326038093250380918403882326
:1017F00019F08FEF9FEF06C080912503909126038B
:1018000088559240909389008093880080E49CE9F9
:101810009093080180930701809184009091850046
:101820008097D0F30E947E0B80918503811105C0C3
:101830008091060181500E94690B1092860327C097
:101840008FEF9FEF06C08091250390912603885566
:1018500092409093890080938800809184009091B9
:1018600085008097D0F30E947E0B809185038111C3
:1018700004C080918603811106C0809186038F5F2A
:101880008093860304C081500E94690BF6CFFF91BC
:10189000EF91CF91BF91AF919F918F917F916F9178
:1018A0005F914F913F912F910F900FBE0F901F901E
:1018B000189524E0829FC00111248C30910538F0E6
:1018C000853F23E0920728F084EF93E008958CE0B1
:1018D00090E00895CF93DF93C0910904C03390F452
:1018E0008C2F807339F0803141F480918703829589
:1018F000807F05C080918C0302C080918D03CF70E2
:10190000D0E015C0CF33E0F4CF70D0E080918703F2
:101910008295807F0E94590CDE01AA0FBB1FA35F36
:10192000BE4F11969C938E93219680918D030E94B9
:10193000590CFE01EE0FFF1FE35FFE4F9183808382
:10194000DF91CF91089580918803909189039F77CB
:101950000E940D03809387038F3029F480918D03BB
:101960008695805804C099E0899F802D112480932A
:101970008C03F8940E946A0C78948091FB03813266
:10198000E1F480918C039FEF980F9E3F78F0809157
:10199000B0008F7D8093B00061E080918C03811155
:1019A00001C060E083E00E945C1C08958093B40055
:1019B0008091B00080628093B0000895FF920F93F1
:1019C0001F93CF93DF930BEF13E0C0E0D0E0B3E0C1
:1019D000FB2E8C2FD801ED918D019E2F907F9031A1
:1019E000F1F4EF70F0E0EE0FFF1FE35FFE4F208198
:1019F00031816F2D0E943D20E92FF0E0EE0FFF1F97
:101A0000E057FD4F61E0808191818217930708F0D4
:101A100060E0FE01E256FD4F80810E945C1C219631
:101A2000CD30D105B1F6CDB7DEB7E5E00C94C720D7
:101A30000F931F93CF93DF9303E613E0C0E0D0E052
:101A400020910904822F8F7090E0C817D907E9F020
:101A50000196C817D90711F42033B8F4F801808132
:101A600091819F70892B79F0F894F80180819181A0
:101A70009F700E94C102FE01EE0FFF1FE35FFE4F49
:101A80009183808378940E94DE0C21960E5F1F4F15
:101A9000C031D105A9F6DF91CF911F910F91089523
:101AA000FF920F931F93CF93DF9381ED93E00E94FA
:101AB000B9018093060190910904292F2F702813F2
:101AC00004C081E0820F8093060190539F3060F440
:101AD0004091060130E0842F90E0019728173907E4
:101AE00019F44F5F4093060180910601813118F08F
:101AF00080E180930601ECE2F3E0DF0112971C9293
:101B0000DF0111971C921082339683E0E335F807CA
:101B1000A1F74FEF3FEFADEAB2E00BEF13E02FEF8D
:101B2000E80189918E018031F8F490E0FD0132974F
:101B30006081FC01EE0FFF1FE80FF91FE65DFC4F0F
:101B40008081862B8083CD010197EC0158818181B2
:101B5000852B81839C918281892B8283609550950E
:101B600090952923352346231396D4E008301D078A
:101B7000B9F6409327033093280320932903CEE935
:101B8000D2E00BEF13E0F12CF80181918F0182324A
:101B900030F08632B8F0863211F460E010C0FBE01D
:101BA000FF1204C08091C1008F7E06C08CE0F81245
:101BB00005C08091C100877F8093C10061E088816A
:101BC0000E94231CF3942196EDE0FE12DDCF80915C
:101BD0000004803231F461E089E00E945C1C82E8FC
:101BE00001C082E08093800081E080938503809330
:101BF00084038091FB03813211F08732D9F461E0D4
:101C000083E00E94231C60E083E00E945C1C8091C2
:101C1000FB03813231F481E08093B0008093B10006
:101C200009C082E08093B00085E08093B1008EE32C
:101C30008093B3008AE1809381008FEF9FEF9093B0
:101C400089008093880080ED97E0909387008093CF
:101C5000860080E49CE990930801809307019093AB
:101C60002603809325031092860380916F00816084
:101C700080936F008091080483FF0DC080916303FF
:101C8000909164039F70892B31F00E94180D10927F
:101C9000840310928503CDB7DEB7E5E00C94C7202E
:101CA000CF93C82F809103048B3221F46C2F8CE0EA
:101CB0000E945C1C8091FB03873249F48091B00044
:101CC000CC2311F0806101C08F7E8093B000CF9152
:101CD0000895A2E2B0E0EFE6FEE00C949E206B01D6
:101CE0007C010E945F1B4B015C0181E00E94720439
:101CF00083E08093CE030E94700566EC71E082E27F
:101D000094E00E942D1D7BE1272EE0E53E2EF7E4B6
:101D10007F2EA6E44A2EB5E55B2EC114D104E10462
:101D2000F10469F00E945F1B681979098A099B090F
:101D30006C157D058E059F0510F080E0D4C0809164
:101D4000CE03843051F764ED71E082E294E00E94AA
:101D50002D1D8FE70E9459030E946C038AA38236CF
:101D600001F501ED13E00E946C03D8018D938D0104
:101D7000B3E00A3F1B07B9F78091D103883309F01C
:101D8000ACC06DED71E082E294E00E942D1D82E412
:101D90008AA361E0CE0182960E94CF052D9A81E050
:101DA000A2C0803741F0893611F581E00E947908A0
:101DB00089E4898304C03982C12CD12C76019091A9
:101DC000CD0380910804992311F0806801C08F77BA
:101DD00080930804EAEFF3E0DE011296822D019071
:101DE0000D928A95E1F76CE1CE01019674C08437BB
:101DF000D9F4E4E5E98383E08A8380E88B838DE08E
:101E00008C838D838AE1EDE2F1E0DE01169601908C
:101E10000D928A95E1F76FE1CE0101960E94CF0500
:101E2000C12CD12C760159C0853789F40AEF13E013
:101E30000E946C03D8018D938D01B4E005311B071E
:101E4000B9F761E080E00E94CB075AA241C0863614
:101E5000B9F44982E3E6F3E0AE014D5F5F4F2081C4
:101E600031813296CA010197DC013C93DA012C934F
:101E70004E5F5F4FB3E0E338FB0789F761E2B4CF11
:101E80008736C9F403E613E00E946C03682E0E94B3
:101E90006C03262D30E0322F2227280F311DF80148
:101EA000219331938F01F3E003381F0769F77AA27A
:101EB0000E9465080DC0873481F4E3E6F3E01192D7
:101EC000119283E0E338F807D1F70E9465087AA2FF
:101ED00061E0CE0182960E94CF0583E08093CE031D
:101EE0000E944D051ACFA296E2E10C94BA201F93EE
:101EF000CF93DF93C82FD62F61E00E94231C61E0AF
:101F00008C2F0E945C1C61E08D2F0E945C1C8AE07B
:101F100090E00E94B41B8D2F0E948F1C892B71F0C2
:101F200060E08C2F0E945C1C8AE090E00E94B41B51
:101F30008D2F0E948F1C11E0892B09F010E060E0CA
:101F40008C2F0E94231C60E08C2F0E945C1C60E0A0
:101F50008D2F0E945C1C812FDF91CF911F910895DE
:101F600080E48093BA001092BD008DE990E09093D8
:101F7000C6038093C5031092600315E004E0C2E03D
:101F8000FC2E80916003813039F480E00E9472045D
:101F9000F09260034398F5CFC0916003C33061F4C1
:101FA0002D988091A2030E949403C093CE030E94B7
:101FB0004D0500936003E5CF80916003843009F7FD
:101FC0008091CE038430E9F68FE70E945903C0E187
:101FD000D3E0E091F903E770F0E0EA56FD4F80812D
:101FE00090E09E01205133402817390724F40E94C5
:101FF0006C038993EECF109360032D9AC2CFAAE2AF
:10200000B0E0E5E0F0E10C94AD201FEF198389E228
:10201000E1EDF3E0DE01129601900D928A95E1F771
:1020200021E04AE2BE016F5F7F4F80E20E94560AC4
:1020300081110EC021E041E0BE016F5F7F4F80E261
:102040000E94AB0A811104C082E08093600302C049
:102050001093600380916003823051F00E945F1BF7
:1020600060935C0370935D0380935E0390935F03C2
:10207000AA96E3E00C94C920A1E0B0E0E2E4F0E12C
:102080000C94AE20809160038230D9F48091A20339
:10209000805A898321E041E0BE016F5F7F4F80E27B
:1020A0000E94560A882369F08FEF809360030E9494
:1020B0005F1B60935C0370935D0380935E0390935A
:1020C0005F032196E2E00C94CA20A1E0B0E0EBE6C9
:1020D000F0E10C94AE20809160038230D1F421E0D5
:1020E00041E0BE016F5F7F4F80E20E94AB0A882310
:1020F00071F08FEF809360030E945F1B60935C031D
:1021000070935D0380935E0390935F0302C08981A7
:1021100001C08FEF2196E2E00C94CA20A2E2B0E069
:10212000E4E9F0E10C949E209E012F5F3F4F80E197
:10213000D9011D928A95E9F768EE71E082E294E098
:1021400029A33AA30E942D1D0E9470051D8A1E8A94
:102150001F8A188E312C212C00E0812C912C5401E7
:1021600080EC482E8DE9582E88E5682E85E3782E80
:1021700090E5C92E93ECD92EE12CF12C84EF91E05F
:10218000A0E0B0E08D8F9E8FAF8FB8A380EC97EF6B
:10219000AAEBB7E3898F9A8FAB8FBC8F80EC9DE958
:1021A000A8E5B5E3898B9A8BAB8BBC8B82E294E07C
:1021B0000E94F91D892B09F4E1C082E294E00E949B
:1021C000261E9C0133272C32310509F442C0ACF4A1
:1021D0002332310509F0ABC019821A821B821C829E
:1021E0001D821E821F82188619861A861B861C86EF
:1021F0001D861E861F86188A60C02434310529F08A
:102200002335310509F4B2C092C064E482E294E05F
:102210000E94111D2AE030E040EC5DE968E575E3BD
:1022200082E294E00E948D1D6CE282E294E00E94C2
:10223000111D2AE030E040EC57EF6AEB77E382E2D1
:1022400094E00E948D1D6CE282E294E00E943F1DAA
:10225000ADCF0F5F043009F0A9CF29813A814B81BE
:102260005C81A8EEB3E00E941A20698B7A8B8B8B7D
:102270009C8B2D813E814F8158850E941A20698F49
:102280007A8F8B8F9C8F29853A854B855C852D8F26
:102290003E8F4F8F58A32D853E854F8558890E94CC
:1022A0001A206B017C0160323EE4730781059105C1
:1022B00030F462E38CE10E94810300E077CF603369
:1022C00045E774078105910510F462E2F3CF6034AD
:1022D0005CE975078105910510F466E2EBCF80E5B6
:1022E000C81683ECD806E104F10410F462E1E2CFF1
:1022F00090E6C9169AEED906E104F10410F465E1FE
:10230000D9CFA0E7CA16A1E1DA06A1E0EA06F104F6
:1023100010F461E0CFCFB0EACB16B6E8DB06B1E04F
:10232000EB06F10410F463E0C5CF65E0C3CF10ED18
:10233000180F1A3008F03ACFE1E0F0E0EC0FFD1F83
:1023400024E0029FE00DF11D1124208131814281A2
:102350005381AAE0B0E00E941A20610F711D811D17
:10236000911D608371838283938320CF49885A882B
:102370006B887C88812C912C540118CF8114910496
:10238000A104B10489F4C301B2010E94070461E011
:1023900070E080E090E00E948E1B1D8A1E8A1F8ADA
:1023A000188E312C22242A948D8D9E8DAF8DB8A14C
:1023B00088169906AA06BB06D0F40E94AA032D89A6
:1023C0003E894F89588D280F311D411D511D2D8B80
:1023D0003E8B4F8B588F381608F4382E821508F430
:1023E000282E3FEF831A930AA30AB30A56C0C301EB
:1023F000B20128EE33E040E050E00E945D20BA01D7
:10240000A9012AE030E082E294E00E94DB1D6CE248
:1024100082E294E00E94111D4AE050E0632D82E2C6
:1024200094E00E94EA1D6CE282E294E00E94111D99
:102430006D897E898F89988DA50194010E945D2008
:10244000BA01A9012AE030E082E294E00E94DB1D9B
:102450006CE282E294E00E94111D4AE050E0622D9D
:1024600082E294E00E94EA1D6CE282E294E00E9423
:102470003F1D4C0C5D1C6E1C7F1C898D9A8DAB8D95
:10248000BC8D84159505A605B70520F449885A88A2
:102490006B887C88812C912C540129893A894B893D
:1024A0005C89283E33404105510509F07FCEA29654
:1024B000E2E10C94BA20A1E0B0E0E1E6F2E10C9494
:1024C000AE2080E00E949F0161E08DE00E94231C0D
:1024D00061E081E10E94231C0E94760160E080E0BF
:1024E0000E94231C61E081E00E94231C40E052EC2A
:1024F00061E070E082E294E00E94411F0E94B70810
:102500000E946A0865EF71E082E294E00E940E1D6D
:1025100080E893E00E9474076CE072E082E294E04D
:102520000E940E1D4AE050E063E070E082E294E019
:102530000E94C31D0E948B017894439A67E086E055
:102540000E94770F882329F043982D980E948E10BF
:10255000FBCF65E083E00E94770F811104C00E94E9
:102560005308811119C06FE472E082E294E00E9486
:102570000E1D60E070E0CB010E94690E882349F0D7
:102580000E94600864E172E082E294E00E942D1DE6
:102590002D9A0E94500D10C00E94500D809104048D
:1025A000823209F0CAC080910504833209F0C5C0A7
:1025B0008091080481FDC7C080910404823231F506
:1025C00080910504833211F581E00E94C108809159
:1025D000080482FF08C06FE272E082E294E00E9489
:1025E0002D1D0E94B00F64E170E080E090E00E9439
:1025F0008E1B21E041E0BE016F5F7F4F80E20E94B1
:10260000AB0A811103C081E0809360036AE372E04A
:1026100082E294E00E940E1D8FE00E949F0180E004
:102620000E9472041092A20380E00E94940380E052
:10263000883170F08093E40283E08093CE030E949F
:10264000700580916003882371F00E94FF0F0BC01A
:1026500021E0280FE82FF0E0EF52FC4F97859923F7
:1026600049F3822FE5CF80910704982F9D7F983200
:1026700029F440E052EC61E070E027C0893271F447
:1026800040EA56E861E070E082E294E00E94411F77
:102690008091C20080628093C2001BC08091F903C8
:1026A0008871803129F440E855E260E070E00DC0A7
:1026B0004091D2035091D3036091D4037091D5031C
:1026C0004A3051056105710570F382E294E00E9481
:1026D000411F82E294E00E94F91D892B29F082E2D9
:1026E00094E00E94261EF5CF80910604843229F0E2
:1026F0008091C1008F7E8093C10080910704853254
:1027000041F08852833028F08091C100877F809308
:10271000C1001092E6021092E502109262030E943C
:102720006B1B60939E0370939F038093A003909311
:10273000A1032196E2E00C94CA20809108048B7FCB
:102740008093080435CF82FD37CF64EF71E080E0DD
:1027500090E00E94690E882309F42ECF0E94600841
:1027600064E172E082E294E00E942D1D0E94500D0F
:102770002D9A22CFCF93DF9382E294E00E94F91D3D
:10278000892BE9F0C091E502D0E0CE0101968F716E
:1027900099272091E60230E08217930781F082E2C8
:1027A00094E00E94261EC951DD4F88838091E50286
:1027B00090E001968F7199278093E502DDCFDF913C
:1027C000CF910895A0E0B0E0E8EEF3E10C94A820EA
:1027D000D82FC62F0E946B1B0091BB031091BC0326
:1027E0002091BD033091BE036B017C01C01AD10A58
:1027F000E20AF30A9701860141E1C41647E2D406D2
:10280000E104F10408F4D1C16093BB037093BC03ED
:102810008093BD039093BE0380910D0190910E01B2
:10282000880F991F8093A303892F87702091A40399
:10283000287F282B2093A40380910F0190911001F1
:10284000880F991F382F330F330F330F2770232B27
:102850002093A403282F2295269527708091A50305
:10286000807C9770990F990F990F822B892B8093F9
:10287000A5032091110130911201220F331F922FD5
:102880009295990F990F907C8F73892B8093A50354
:10289000932F9295990F990F907C822F869586950C
:1028A000892B8093A60332FB882780F92091A70308
:1028B0002E7F282B2093A703809113019091140160
:1028C000880F991F382F330F2170232B2093A703D4
:1028D000382F331F3327331F2091A803207F892FE0
:1028E0008770880F232B282B2093A8038091150134
:1028F00090911601880F991F382F3295307F2F70D5
:10290000232B2093A803382F32953F702091A903E1
:102910002078892F87708295807F232B282B209306
:10292000A9038091170190911801880F991F2F77A3
:102930002093A903292F2795222727958695822B57
:102940008093AA03892F869583702091AB032C7FF7
:10295000282B2093AB038091190190911A01880FC5
:10296000991F382F330F330F2370232B2093AB0382
:10297000382F32953695369533702091AC03207EF2
:10298000892F8770880F880F232B282B2093AC0367
:1029900080911B0190911C01880F991F382F32954F
:1029A000330F307E2F71232B2093AC039295990F18
:1029B000907E869586958695892B8093AD03809130
:1029C0001D0190911E01880F991F8093AE03892FDE
:1029D00087702091AF03287F282B2093AF0380912D
:1029E0001F0190912001880F991F382F330F330F4B
:1029F000330F2770232B2093AF03282F2295269582
:102A000027708091B003807C9770990F990F990F70
:102A1000822B892B8093B0032091210130912201D8
:102A2000220F331F922F9295990F990F907C8F73DD
:102A3000892B8093B003932F9295990F990F907CD7
:102A4000822F86958695892B8093B10332FB882748
:102A500080F92091B2032E7F282B2093B20380911E
:102A6000230190912401880F991F382F330F217073
:102A7000232B2093B203382F331F3327331F20918A
:102A8000B303207F892F8770880F232B282B209357
:102A9000B3038091250190912601880F991F382F4B
:102AA0003295307F2F70232B2093B303382F32952C
:102AB0003F702091B4032078892F87708295807FA2
:102AC000232B282B2093B403809127019091280178
:102AD000880F991F2F772093B403292F279522273A
:102AE00027958695822B8093B50396959370809158
:102AF000B6038C7F892B8093B603209129013091F6
:102B00002A01220F331F922F990F990F8370892B5F
:102B10008093B60322952695269523708091B7035E
:102B2000807E932F9770990F990F822B892B80931A
:102B3000B70320912B0130912C01220F331F922FCC
:102B40009295990F907E8F71892B8093B703832F75
:102B50008295880F807E269526952695282B209392
:102B6000B803DD2311F088E001C080E0CC2311F030
:102B700094E001C090E0892B8093B9036FE070E08E
:102B800082E294E00E940201C3EAD3E0699182E20A
:102B900094E00E94531E83E0CA3BD807B9F760E077
:102BA00070E082E294E00E940201CDB7DEB7E8E077
:102BB0000C94C420CF93C82F682F82E294E00E9427
:102BC000531E8C2F0E940A01CF910895A0E0B0E01F
:102BD000ECEEF5E10C94A820C82F0E946B1B00912D
:102BE000BB031091BC032091BD033091BE036B0168
:102BF0007C01C01AD10AE20AF30A9701860141E179
:102C0000C41647E2D406E104F10408F445C0609319
:102C1000BB037093BC038093BD039093BE031092DB
:102C2000D0031092CF0388EA0E94DA15CC2311F06A
:102C300081E801C081E00E94DA1580E10E94DA1586
:102C400000E010E0F801EE0FFF1FE35FFE4F808110
:102C500091810E94EC02EC01B3E0CC0FDD1FBA952C
:102C6000E1F78D2F0E94DA158C2F0E94DA150F5F85
:102C70001F4F0031110531F76091D00370E082E2FF
:102C800094E00E94FA006091CF037091D0037727FF
:102C900082E294E00E94FA00CDB7DEB7E8E00C943F
:102CA000C420AAE1B0E0E7E5F6E10C94A0200E9480
:102CB0009B008CE00E947B0381110BC068E872E0EE
:102CC00082E294E00E942D1D80E00E9472040E9426
:102CD00070050E94BA130E946B1B0E94651091E060
:102CE000853009F090E01FEF8091CE03843009F425
:102CF000FEC19111FCC17CC00E94AE0390938B0376
:102D000080938A032D9AC0929E03D0929F03E092F3
:102D1000A003F092A1031092610380918803909127
:102D20008903880F991F816090938903809388039A
:102D3000439880E00E94500E80911003982F9E735C
:102D400009F02CC2F8948091F90341E153E06DE061
:102D500071E087700E943B020E946A0C7894909107
:102D6000100380915A0390FF13C2811124C093E68F
:102D7000E92E93E0F92E00E010E0F70180819181C7
:102D800094FD0CC0F801EE0FFF1FE35FFE4F808142
:102D900091810E94EC02D7018D939C930F5F1F4F8E
:102DA000B2E0EB0EF11C0031110539F70E94650805
:102DB00081E080935A0380916203811103C081E016
:102DC0008093620310928303109285031092840310
:102DD0008091F903887109F009C20E94DE0C83E03A
:102DE0008093CE030E944D0581E080935B032D9874
:102DF0000E946B1B4B015C010E945F1B6B017C01FD
:102E000080916103823008F063C040909E0350902F
:102E10009F036090A0037090A10380919A0390910A
:102E20009B03A0919C03B0919D0384159505A60575
:102E3000B70509F44DC081ED93E00E94C9016C5DB6
:102E40007540810991099501840104191509260924
:102E500037096017710782079307D0F540929A03EC
:102E600050929B0360929C0370929D030E94AA0360
:102E7000282F80938E0380918F0390919003820F6F
:102E8000911D9093900380938F03609191036F5FE6
:102E9000609391036930E0F070E00E9449207093E4
:102EA000900360938F0380918D03E3E08E9F600D0C
:102EB000711D1124769567957695679560938D03BE
:102EC0000E94A30C1092900310928F031092910312
:102ED000809162030091E402882351F11091610313
:102EE000101708F029C240909E0350909F036090F5
:102EF000A0037090A103A501940124193509460986
:102F000057092F8B388F498F5A8F81ED93E00E949C
:102F1000C90168517C4F8F4F9F4F2F89388D498D44
:102F20005A8D621773078407950708F4CCC104C251
:102F300080919E0390919F03A091A003B091A10363
:102F400075016401C81AD90AEA0AFB0A81ED93E007
:102F50000E94C9019B01AC01A02FB0E00E941A2081
:102F60006C157D058E059F0558F480929E03909206
:102F70009F03A092A003B092A10381E080935B0322
:102F800080918403811116C080910704883219F45E
:102F90000E94020B0FC0893239F460916103809165
:102FA00083030E94E21306C08A3221F480918303D6
:102FB0000E94E61580915B03882309F472C0E091BA
:102FC000A203EF5FE093A203E83131F0F0E0EF52AB
:102FD000FC4F8785811102C01092A20380910A04E0
:102FE00090910B04A0910C04B0910D04892B8A2BB5
:102FF0008B2B09F44EC08091920390919303A09182
:103000009403B0919503892B8A2B8B2B09F441C033
:103010000E946006082F10E02091090130910A01FA
:1030200036952795369527952C5E3F4F201731070B
:1030300070F40E945F1B68517C4F8F4F9F4F6093CD
:103040009203709393038093940390939503C80124
:10305000880F991F880F991F4091090150910A010B
:103060009A01220F331F240F351F820F931F96954D
:1030700087959695879590930A01809309016091B1
:10308000D6037091D7038091D8039091D9030E9401
:1030900007048091A2030E9494030E943C101092A6
:1030A0005B03809160038F3F09F041C20E945F1B68
:1030B00000915C0310915D0320915E0330915F03EA
:1030C000601B710B820B930B693E73408105910568
:1030D00008F42DC20E945F1B60935C0370935D0334
:1030E00080935E0390935F030E94FF0F20C20E94B3
:1030F0006B1B6B017C018091CE038430D1F48FE790
:103100000E94590300E113E0E091F903E770F0E059
:10311000EA56FD4F808190E09801205133402817F6
:1031200039070CF0E9CD0E946C03D8018D938D0115
:10313000EBCFE091F903E770F0E0EA56FD4F4081F4
:103140004F5F21E0BE016F5F7F4F80E20E94AB0ABC
:10315000882371F0109360030E945F1B60935C03EF
:1031600070935D0380935E0390935F0390E0BCCD0A
:10317000E091F903E770F0E0EA56FD4F408150E03E
:10318000BE016E5F7F4F80E193E00E94DB20BBCDEC
:10319000882309F410CE10925A030DCE982F9873FD
:1031A000983309F008CE90910703892787FF03CE53
:1031B00090589093070380910704853209F0FBCD66
:1031C00010E0212F30E080911003877090E082178B
:1031D00093070CF4F0CD1F5FE12FF0E0E05FFC4FB0
:1031E000608182E294E00E94531EEBCF809107033E
:1031F00090911003982796FD5AC0807C90E489270F
:10320000809307038091E6023091E5028317D1F0A5
:10321000E8E0F3E020E02F5F90E0DC01A951BD4F32
:103220004C91419301968F719927283011F08313A7
:10323000F2CF8093E602295C80910703282B20932C
:10324000070335C080918E038093080380910404A6
:10325000863251F482E10E94B81C95958795959528
:1032600087958093090302C0109209038091050499
:10327000863251F483E10E94B81C95958795959507
:10328000879580930A0302C010920A0380918A03F3
:1032900090918B0390930B0380930C038091880390
:1032A000909189039F770E940D0380930D0369E03D
:1032B00087E093E00E9488050E94F70581118DCD7B
:1032C0000E94BA13F9CF8091880390918903880FE7
:1032D000991F909389038093880381E080935B0317
:1032E000111110C0C0929603D0929703E0929803F8
:1032F000F092990310929203109293031092940308
:10330000109295031F5F1093610381ED93E00E947B
:10331000C901640D751D861D971D60939E037093F2
:103320009F038093A0039093A103439A81E00E949E
:10333000500E0E94A30C03C0101709F4A7C080917F
:103340006103882309F41CCE809112048823D9F0EC
:1033500090918303911117C0409196035091970368
:10336000609198037091990346015701841A950A58
:10337000A60AB70A90E00E942301681579058A051C
:103380009B0508F4B5C0809114048823D9F090916E
:103390008503911117C04091960350919703609156
:1033A00098037091990346015701841A950AA60A59
:1033B000B70A90E00E942301681579058A059B05EC
:1033C00008F4ADC0809113048823D9F09091840350
:1033D000911117C040919603509197036091980303
:1033E0007091990346015701841A950AA60AB70AF3
:1033F00090E00E942301681579058A059B0508F471
:1034000092C080910A0490910B04A0910C04B09199
:103410000D04892B8A2B8B2B09F4B2CD809192035A
:1034200090919303A0919403B09195030097A10507
:10343000B10509F4A5CDC81AD90AEA0AFB0AF7FCB6
:103440009FCD80910804829581700E94A30680E040
:103450000E9472040E944D050E945F1B6B017C015B
:1034600020910F0430E0A8EEB3E00E940B20C60EBE
:10347000D71EE81EF91E6894C0F8C0929203D0923D
:103480009303E0929403F09295037ACD80919E038A
:1034900090919F03A091A003B091A1032401350155
:1034A000481A590A6A0A7B0A81ED93E00E94C90111
:1034B0009B01AC01A12FB0E00E941A206415750594
:1034C0008605970508F03BCF109289031092880378
:1034D00081E080935B0310928D030E94A30C809285
:1034E0009E0390929F03A092A003B092A10327CFC6
:1034F00081E0809383030E94180D80910E040E9446
:1035000048016C0D7D1D8E1D9F1D616060939203AF
:1035100070939303809394039093950334CF81E049
:10352000809385034FCF81E0809384036ACF6A96AE
:10353000E0E10C94BC208230E8F4E82FF0E0EE0FDC
:10354000FF1FEB5EFB4F71836083813041F0809100
:1035500069008C7F842B80936900E89A089580919C
:103560006900440F551F440F551F837F842B8093A0
:103570006900E99A08951F920F920FB60F921124D5
:103580002F933F934F935F936F937F938F939F936B
:10359000AF93BF93EF93FF9380911504909116041E
:1035A000892B29F0E0911504F09116040995FF91FB
:1035B000EF91BF91AF919F918F917F916F915F91AB
:1035C0004F913F912F910F900FBE0F901F90189524
:1035D0001F920F920FB60F9211242F933F934F9388
:1035E0005F936F937F938F939F93AF93BF93EF936B
:1035F000FF938091170490911804892B29F0E09192
:103600001704F09118040995FF91EF91BF91AF91C4
:103610009F918F917F916F915F914F913F912F91EA
:103620000F900FBE0F901F9018951F920F920FB61C
:103630000F9211242F933F938F939F93AF93BF9338
:1036400080911A0490911B04A0911C04B0911D0458
:103650003091190423E0230F2D3720F40196A11D8A
:10366000B11D05C026E8230F0296A11DB11D2093B0
:10367000190480931A0490931B04A0931C04B09324
:103680001D0480911E0490911F04A0912004B0910C
:1036900021040196A11DB11D80931E0490931F0467
:1036A000A0932004B0932104BF91AF919F918F917B
:1036B0003F912F910F900FBE0F901F9018952FB72D
:1036C000F89460911A0470911B0480911C049091ED
:1036D0001D042FBF08953FB7F89480911E04909168
:1036E0001F04A0912004B091210426B5A89B05C019
:1036F0002F3F19F00196A11DB11D3FBF6627782FFE
:10370000892F9A2F620F711D811D911D42E0660F56
:10371000771F881F991F4A95D1F70895CF92DF929E
:10372000EF92FF92CF93DF936B017C010E946B1BA2
:10373000EB01C114D104E104F10479F00E946B1B88
:103740006C1B7D0B683E7340A0F381E0C81AD10862
:10375000E108F108C851DC4FECCFDF91CF91FF9029
:10376000EF90DF90CF9008950197009739F0880F80
:10377000991F880F991F02970197F1F70895789480
:1037800084B5826084BD84B5816084BD85B5826066
:1037900085BD85B5816085BDEEE6F0E08081816004
:1037A0008083E1E8F0E01082808182608083808104
:1037B00081608083E0E8F0E0808181608083E1EBDC
:1037C000F0E0808184608083E0EBF0E080818160C4
:1037D0008083EAE7F0E0808184608083808182607A
:1037E0008083808181608083808180688083109263
:1037F000C1000895833081F028F4813099F082303F
:10380000A1F008958630A9F08730B9F08430D1F462
:10381000809180008F7D03C0809180008F7780939E
:103820008000089584B58F7702C084B58F7D84BDF4
:1038300008958091B0008F7703C08091B0008F7D94
:103840008093B0000895CF93DF9390E0FC01E4589B
:10385000FF4F2491FC01E057FF4F8491882349F1E9
:1038600090E0880F991FFC01E854FF4FA591B49197
:1038700082559F4FFC01C591D4919FB7611108C03B
:10388000F8948C91209582238C93888182230AC09E
:10389000623051F4F8948C91322F309583238C93BD
:1038A0008881822B888304C0F8948C91822B8C931E
:1038B0009FBFDF91CF910895A1E0B0E0E2E6FCE187
:1038C0000C94AC20282F30E0F901E859FF4F849187
:1038D000F901E458FF4F1491F901E057FF4F0491AB
:1038E0000023C9F0882321F069830E94FA1B6981B3
:1038F000E02FF0E0EE0FFF1FE255FF4FA591B491CE
:103900009FB7F8948C91611103C01095812301C079
:10391000812B8C939FBF2196E4E00C94C820CF9319
:10392000DF93282F30E0F901E859FF4F8491F90126
:10393000E458FF4FD491F901E057FF4FC491CC23D5
:1039400091F081110E94FA1BEC2FF0E0EE0FFF1FA7
:10395000EC55FF4FA591B4912C912D2381E090E07F
:1039600021F480E002C080E090E0DF91CF910895E3
:103970008E3008F08E5087702091B90190E4299F15
:1039800090011124822B80937C0080917A008064C6
:1039900080937A0080917A0086FDFCCF8091780038
:1039A0002091790090E0922B0895A0E0B0E0EBED3B
:1039B000FCE10C94A8206C017A01EB01E60EF71EE5
:1039C00000E010E0CE15DF0561F06991D601ED91C0
:1039D000FC910190F081E02DC6010995080F191F97
:1039E000F1CFC801CDB7DEB7E8E00C94C420611573
:1039F000710589F0DB010D900020E9F7AD01415020
:103A00005109461B570BDC01ED91FC910280F381BB
:103A1000E02D0995089580E090E008950E94F71C3C
:103A20000895DC01ED91FC910190F081E02D099564
:103A300008950F931F93CF93DF93EC016DE00E94E5
:103A4000111D8C016AE0CE010E94111D800F911F93
:103A5000DF91CF911F910F9108950F931F93CF93F3
:103A6000DF93EC010E94F71C8C01CE010E94191D0E
:103A7000800F911FDF91CF911F910F9108950F93A8
:103A80001F93CF93DF93EC010E94111D8C01CE0197
:103A90000E94191D800F911FDF91CF911F910F91EF
:103AA0000895A1E2B0E0E7E5FDE10C94A4207C01DB
:103AB000C42EE52FCB01D22E19A221E02D1510F036
:103AC0002AE0D22E8E010F5D1F4F8D2C912CA12C40
:103AD000B12C6C2D7E2FA50194010E945D208C2DB0
:103AE000D29E80191124015011098A3010F4805D92
:103AF00001C0895CF801808321153105410551051C
:103B000021F0C22EE32FCA01E4CFB801C7010E9401
:103B1000F71CA196ECE00C94C020A0E0B0E0E3E933
:103B2000FDE10C94A820EC016A017B01211531050F
:103B300041F4E881F9810190F081E02D642F09952D
:103B40001DC02A303105A9F477FF12C06DE20E9432
:103B5000111D8C0144275527BA014C195D096E09C6
:103B60007F092AE0CE010E94511D800F911F06C0DF
:103B70002AE0B701A601CE010E94511DCDB7DEB7E4
:103B8000E8E00C94C4200F931F93CF93DF93EC01D4
:103B90009A01AB01662757FD6095762F0E948D1D17
:103BA0008C01CE010E94191D800F911FDF91CF91D2
:103BB0001F910F9108952115310549F4DC01ED9114
:103BC000FC910190F081E02D642F099508950E94E9
:103BD000511D08959A01462F50E060E070E00E9468
:103BE000DB1D08959A01AB0160E070E00E94DB1DCF
:103BF0000895FC0124853585F901E05CFF4F808143
:103C00009181F901EE5BFF4F20813181821B930B83
:103C10008F7399270895FC0184859585FC01E05CEC
:103C2000FF4F40815181FC01EE5BFF4F20813181CC
:103C30004217530741F00190F081E02DE80FF91F82
:103C4000808190E008958FEF9FEF0895FC018485B7
:103C50009585FC01E05CFF4F40815181FC01EE5BEA
:103C6000FF4F208131814217530779F0A081B18144
:103C7000A80FB91F8C91208131812F5F3F4F2F7387
:103C800033273183208390E008958FEF9FEF0895CD
:103C9000FC0181A1882329F0A489B5898C9186FF34
:103CA000FBCF11A20895CF93DF93FC0126853785C2
:103CB000D901A05CBF4F8D919C91119701968F7394
:103CC0009927E901CE5BDF4F488159818417950719
:103CD000D9F30D90BC91A02DA20FB31F6C93A685B4
:103CE000B785A05CBF4F11969C938E93A689B78928
:103CF0002C9181E090E0078C02C0880F991F0A94F4
:103D0000E2F7282B2C9381E081A30488F589E02D2C
:103D100080818064808381E090E0DF91CF9108957D
:103D200008951F920F920FB60F9211242F933F9375
:103D30004F938F939F93EF93FF938091C00082FDE9
:103D40001CC04091C6008091C8049091C90401969E
:103D50008F7399272091CA043091CB04821793075F
:103D600071F0E091C804F091C904E857FB4F40831B
:103D70009093C9048093C80402C08091C600FF914B
:103D8000EF919F918F914F913F912F910F900FBE87
:103D90000F901F90189582E294E00E94F91D892BE4
:103DA00011F00E94901E08951F920F920FB60F926D
:103DB00011242F933F938F939F93EF93FF93209121
:103DC000840430918504809186049091870428179B
:103DD000390731F48091C1008F7D8093C10014C0F8
:103DE000E0918604F0918704EC5BFB4F2081809189
:103DF00086049091870401968F7399279093870486
:103E0000809386042093C600FF91EF919F918F913C
:103E10003F912F910F900FBE0F901F901895A0E02B
:103E2000B0E0E5E1FFE10C94A420FC0113821282D2
:103E300088EE93E0A0E0B0E084839583A683B78307
:103E400086ED92E0918380837587648757874687E4
:103E5000318B208B138B028BF58AE48AD78AC68A32
:103E6000B18EA08E938E828E8F85848F8889858F68
:103E70008989868F8A89878F8B8980A3ECE00C944F
:103E8000C020CF92DF92EF92FF92CF93DF93EC01AD
:103E90006A017B01411581EE580761057105F9F052
:103EA000EC89FD8981E090E008A002C0880F991F8D
:103EB0000A94E2F7808360E079E08DE390E0A70167
:103EC00096010E945D202150310941095109569502
:103ED000479537952795211580E1380798F0EC89AB
:103EE000FD89108260E874E88EE190E0A7019601F8
:103EF0000E945D202150310941095109569547958D
:103F000037952795E889F9893083EA89FB892083E9
:103F100019A2EE89FF89408181E090E09C010C8C20
:103F200002C0220F331F0A94E2F7422B4083EE892E
:103F3000FF8940819C010D8C02C0220F331F0A941F
:103F4000E2F7422B4083EE89FF8940819C010E8C71
:103F500002C0220F331F0A94E2F7422B4083EE89FE
:103F6000FF8920810F8C02C0880F991F0A94E2F705
:103F7000809582238083DF91CF91FF90EF90DF9037
:103F8000CF9008958F929F92AF92BF92CF92DF927F
:103F9000EF92FF920F931F9381E08F9385E08F93B1
:103FA00087E08F9383E08F9384E08F93E6EC8E2EEF
:103FB000912CF2ECAF2EB12CA1ECCA2ED12CB0EC8E
:103FC000EB2EF12C04EC10E025EC30E044E454E05E
:103FD00068E874E082E294E00E940F1F0F900F9057
:103FE0000F900F900F901F910F91FF90EF90DF9027
:103FF000CF90BF90AF909F908F9008950E94BF1B6D
:104000000E945B12CBECDEE10E9451162097E1F397
:104010000E94CB1EF9CFA29FB001B39FC001A39F06
:10402000700D811D1124911DB29F700D811D1124F1
:10403000911D08950E940B20A59F900DB49F900D97
:10404000A49F800D911D11240895B7FF0C941A2090
:104050000E941A20821B930B0895DB018F939F937C
:104060000E941A20BF91AF91A29F800D911DA39F26
:10407000900DB29F900D11240895991B79E004C012
:10408000991F961708F0961B881F7A95C9F7809597
:104090000895AA1BBB1B51E107C0AA1FBB1FA6178F
:1040A000B70710F0A61BB70B881F991F5A95A9F7E1
:1040B00080959095BC01CD010895A1E21A2EAA1B0E
:1040C000BB1BFD010DC0AA1FBB1FEE1FFF1FA217C8
:1040D000B307E407F50720F0A21BB30BE40BF50BC5
:1040E000661F771F881F991F1A9469F7609570954E
:1040F000809590959B01AC01BD01CF010895052EDF
:1041000097FB1EF400940E94962057FD07D00E9452
:104110005D2007FC03D04EF40C94962050954095FA
:10412000309521953F4F4F4F5F4F08959095809563
:10413000709561957F4F8F4F9F4F08952F923F92BB
:104140004F925F926F927F928F929F92AF92BF92A7
:10415000CF92DF92EF92FF920F931F93CF93DF9353
:10416000CDB7DEB7CA1BDB0B0FB6F894DEBF0FBEB0
:10417000CDBF09942A88398848885F846E847D84FD
:104180008C849B84AA84B984C884DF80EE80FD80FF
:104190000C811B81AA81B981CE0FD11D0FB6F89475
:1041A000DEBF0FBECDBFED010895EE0FFF1F0590DE
:1041B000F491E02D0994FB01DC0102C001900D9205
:1041C00041505040D8F70895F999FECF92BD81BD76
:1041D000F89A992780B50895262FF999FECF1FBA2E
:1041E00092BD81BD20BD0FB6F894FA9AF99A0FBE20
:0841F00001960895F894FFCF39
:1041F8000000CC04200008409CFF00881300020047
:104208000200020002000200020002000200020096
:104218000200020002000200020002000200210067
:10422800270520082B092209260A230A260B240C15
:10423800250C280C290C2A8025000005400AA120FD
:104248004EA50020244EA52C2330C01200001A4091
:104258000AA1204EA5001B1E27522C2330802500C2
:104268000005400AA1204EA50020244EA52C23308D
:10427800004B000006400AD0009D49007B289D495C
:104288002C233000E1000005400A4501D7DC03B8C3
:104298001E0EBF00232E48E801008A400A6001551F
:1042A8005502AD1E20000023C80154582074696DC2
:1042B800656F7574210057616974696E672062695A
:1042C8006E640A00476F7420706B740A006461742E
:1042D8006120676F6F640A007363616E6E65722098
:1042E8006D6F6465004F70656E4C52536E67205257
:1042F80058207374617274696E672000206F6E2095
:104308004857200053617665642062696E642064B2
:1043180061746120746F20454550524F4D0A004921
:1043280020616D20736C61766500456E74657269F5
:104338006E67206E6F726D616C206D6F64650045ED
:104348004550524F4D2064617461206E6F74207621
:10435800616C6964206F722062696E64206A756D91
:1043680070706572207365742C20666F7263696E55
:10437800672062696E640A0052582068616E67009F
:10438800B200F4014C0300070B0C101115000305D3
:10439800060708090A0B0C121300010000080000A8
:1043A800200000400000800100000200000400001E
:1043B80008000010000000100000200000000100AC
:1043C800000200000000531ED51CF91D261E0B1EFE
:0243D800481E7D
:107E00000F92CDB7DEB7112484B714BE81FFF1D035
:107E100082E08093C00088E18093C10086E0809377
:107E2000C20080E18093C4008EE0CDD088249924E4
:107E3000CC24C394F5E0DF2EE1E1EE2E73E0F72EC3
:107E4000B6D0082F813479F4B2D08983C2D0898129
:107E5000823811F481E005C0813811F485E001C059
:107E600083E09ED09AC0823411F484E103C085344B
:107E700019F485E0B6D091C0853561F498D0082F0B
:107E800010E095D090E0982E8824802A912A880CC2
:107E9000991C82C0863521F484E0A3D080E0E1CF34
:107EA000843609F04CC083D082D0A82E80D0B82E62
:107EB00000E011E07CD0F80181938F01AE16D1F77C
:107EC00088D0FB2DF53489F4E0E0F1E00BC0F9999E
:107ED000FECF92BC81BC0894811C911C819180BD15
:107EE000FA9AF99AEA1598F358C08B2D863409F05E
:107EF00054C0F401F7BEE89507B600FCFDCFF401CD
:107F0000A0E0B1E02C9130E011968C91119790E0B7
:107F1000982F8827822B932B12960C01C7BEE895C9
:107F20001124329681E0A038B80761F7F401D7BE7A
:107F3000E89507B600FCFDCFE7BEE8952EC0843774
:107F4000F1F435D034D0182F32D0B82E42D0FB2DDA
:107F5000F63421F4F40105914F010CC0FB2DF534EA
:107F600049F4F999FECF92BC81BC0894811C911C04
:107F7000F89A00B5802F14D0115049F70EC08537FC
:107F800039F427D08EE10CD085E90AD08FE069CF93
:107F9000813511F488E017D01CD080E101D050CF9A
:107FA0009091C00095FFFCCF8093C600089580910A
:107FB000C00087FFFCCF8091C00084FD01C0A89560
:107FC0008091C6000895E0E6F0E098E19083808318
:107FD0000895EDDF803219F088E0F5DFFFCF84E10E
:107FE000DFCF1F93182FE3DF1150E9F7F2DF1F9166
:0E7FF0000895282E80E0E7DFEE27FF27099492
:027FFE0001057B
:0400000300007E007B
:00000001FF
